:100000000C942A001895000018950000189500001F
:10001000189500001895000018950000189500002C
:10002000189500000C94EB0218950000189500003C
:10003000189500001895000018950000189500000C
:1000400018950000189500001895000018950000FC
:10005000189500008FE58DBFC8E3E0E24E2E84E0E6
:100060008EBFD4E0F4E05F2EA89584B7082E877F7A
:1000700084BF88E1992781BD91BDEEEFF3E0A0E652
:10008000B0E088278D933197E9F766248FEF8ABB1C
:100090008FEF81BB8FEF84BBBB98C39A83E083BF94
:1000A000789479B7716079BF83E083BF81E08093F2
:1000B000A300A9EAB0E08C9187FB16F00C947000C5
:1000C0000091A3000D3011F00C946B0081E080933F
:1000D000A3000C947000A3EAB0E08C918F5F8C9326
:1000E00080E08093AA007091A9007F7E7093A900A0
:1000F0000091A300013011F00C94890080E08093FE
:10010000A70083E28093A40081E08093A8000C9470
:100110004A01023011F00C94980085E48093A70006
:1001200085E68093A40084E08093A8000C944A01A3
:10013000033011F00C94A70085E68093A7008DE6AC
:100140008093A4008FE08093A8000C944A010430AF
:1001500011F00C94BB0086E48093A7008CE480939C
:10016000A4008BE08093A8007091A9007061709347
:10017000A9000C944A01053011F00C94CA0083E2E6
:100180008093A70085E48093A40082E08093A80078
:100190000C944A01063011F00C94D9008DE680933E
:1001A000A70083E78093A4008EE08093A8000C94BE
:1001B0004A01073011F00C94E80083E78093A70010
:1001C0008FE88093A40088E08093A8000C944A01F3
:1001D000093011F00C94F7008FE88093A70087EAAC
:1001E0008093A40085E08093A8000C944A010A3013
:1001F00011F00C94060187EA8093A70087EB8093A7
:10020000A40086E08093A8000C944A010B3011F002
:100210000C941A0180E08093A70080E48093A400EE
:1002200085E08093A8007091A90070617093A90087
:100230000C944A010C3011F00C94290187EB809347
:10024000A7008FEB8093A40080E18093A8000C941A
:100250004A01083011F00C9438018FEB8093A7000D
:1002600083EC8093A40080E18093A8000C944A0161
:100270000D3011F00C944A0180E48093A70086E4CD
:100280008093A4008CE08093A8007091A900706115
:100290007093A90080E08093A200A2EAB0E08C9164
:1002A0008F5F8C93A7EAB0E00D91112740E150E0F9
:1002B0000E94811FA5EAB0E00D931C93A5EAB0E06F
:1002C0000D911C91A2EAB0E04D915527040F151F26
:1002D000A5EAB0E00D931C93A5EAB0E00D911C9146
:1002E00001501040A5EAB0E00D931C93A9EAB0E0DC
:1002F0008C9184FB16F40C948F01EEE0F9E0A5EAF2
:10030000B0E08D919C91A2EAB0E0AD90BB24A0E654
:10031000B0E0AA0DBB1D0E949B1F0C949F01EEEC48
:10032000F9E3A5EAB0E08D919C91A2EAB0E0AD902E
:10033000BB24A0E6B0E0AA0DBB1D0E949B1F00914C
:10034000A200003111F00C944D0180E08093A200D6
:10035000A2EAB0E08C918F5F8C93A7EAB0E00D9198
:10036000112740E150E00E94811FA5EAB0E00D9303
:100370001C93A5EAB0E00D911C91A2EAB0E04D916A
:100380005527040F151FA5EAB0E00D931C93A5EAAD
:10039000B0E00D911C9101501040A5EAB0E00D9322
:1003A0001C93A9EAB0E08C9184FB16F40C94EA014A
:1003B000EEE3F5E1A5EAB0E08D919C91A2EAB0E010
:1003C000AD90BB24A0E7B0E0AA0DBB1D0E949B1F0F
:1003D0000C94FA01EEECF9E3A5EAB0E08D919C9162
:1003E000A2EAB0E0AD90BB24A0E7B0E0AA0DBB1D2F
:1003F0000E949B1F0091A200003111F00C94A801F3
:1004000080E08093A200A2EAB0E08C918F5F8C9391
:10041000A7EAB0E00D91112740E150E00E94811F52
:10042000A5EAB0E00D931C93A5EAB0E00D911C91F4
:10043000A2EAB0E04D915527040F151FA5EAB0E0E0
:100440000D931C93A5EAB0E00D911C910150104052
:10045000A5EAB0E00D931C93A9EAB0E08C9184FB6F
:1004600016F40C944502EEE6F1E2A5EAB0E08D91B7
:100470009C91A2EAB0E0AD90BB24A0E8B0E0AA0D48
:10048000BB1D0E949B1F0C945502EEECF9E3A5EAFC
:10049000B0E08D919C91A2EAB0E0AD90BB24A0E8C1
:1004A000B0E0AA0DBB1D0E949B1F0091A20000316D
:1004B00011F00C94030280E08093A200A2EAB0E065
:1004C0008C918F5F8C93A7EAB0E00D91112740E1EA
:1004D00050E00E94811FA5EAB0E00D931C93A5EAAD
:1004E000B0E00D911C91A2EAB0E04D915527040FA8
:1004F000151FA5EAB0E00D931C93A5EAB0E00D919D
:100500001C9101501040A5EAB0E00D931C93A9EA9C
:10051000B0E08C9184FB16F40C94A002EEE9FDE2AD
:10052000A5EAB0E08D919C91A2EAB0E0AD90BB2429
:10053000A0E9B0E0AA0DBB1D0E949B1F0C94B00265
:10054000EEECF9E3A5EAB0E08D919C91A2EAB0E06F
:10055000AD90BB24A0E9B0E0AA0DBB1D0E949B1F7B
:100560000091A200003111F00C945E02A7EAB0E005
:100570008C918F5F8C9384E490E00E94721F409175
:10058000A4000091A700041711F00C944A01AAEAF4
:10059000B0E08C918F5F8C934091A8000091AA00ED
:1005A000041781E009F080E08F93A9EAB0E08C9114
:1005B00086FB81E00EF080E09F91892B882311F467
:1005C0000C9473007091A9007F7B7093A9000C9428
:1005D0005900F894FFCF0F921F922F923F924F92A3
:1005E0005F927F92AF92BF920F931F932F933F938F
:1005F0004F935F936F937F938F939F93AF93BF932B
:10060000CF93DF93EF93FF938FB78F93882783BFA9
:1006100000916000053011F00C94130381E0809389
:1006200060000C941803A0E6B0E08C918F5F8C936F
:1006300080E08093A10070E072BB70E075BB70E059
:100640007BBBA1EAB0E08C918F5F8C93009160003E
:10065000013011F00C944803979AA1EAB0E0AD90F4
:10066000BB24A0E6B0E0AA0DBB1D0C91013010F434
:100670000C9441037091A90070627093A9000C94CE
:1006800046037091A9007F7D7093A9000C94A60386
:10069000023011F00C946803969AA1EAB0E0AD9094
:1006A000BB24A0E7B0E0AA0DBB1D0C91013010F4F3
:1006B0000C9461037091A90070627093A9000C946E
:1006C00066037091A9007F7D7093A9000C94A60326
:1006D000033011F00C948803959AA1EAB0E0AD9034
:1006E000BB24A0E8B0E0AA0DBB1D0C91013010F4B2
:1006F0000C9481037091A90070627093A9000C940E
:1007000086037091A9007F7D7093A9000C94A603C5
:10071000043011F00C94A603949AA1EAB0E0AD90D5
:10072000BB24A0E9B0E0AA0DBB1D0C91013010F470
:100730000C94A1037091A90070627093A9000C94AD
:10074000A6037091A9007F7D7093A9000091A1007C
:10075000093010F00C94ED03A9EAB0E08C9185FB10
:1007600016F00C94EB030091A100013011F00C94F1
:10077000BC03A89A0C94EB03023011F00C94C30351
:10078000A99A0C94EB03033011F00C94CA03AA9AB3
:100790000C94EB03043011F00C94D103AB9A0C943D
:1007A000EB03053011F00C94D803AC9A0C94EB03D6
:1007B000063011F00C94DF03AD9A0C94EB03073074
:1007C00011F00C94E603AE9A0C94EB03083011F090
:1007D0000C94EB03AF9A0C942C04A9EAB0E08C9132
:1007E00085FB16F00C942C040091A100093011F047
:1007F0000C94FD03D89A0C942C040A3011F00C943C
:100800000404D99A0C942C040B3011F00C940B04B2
:10081000DA9A0C942C040C3011F00C941204DB9A2C
:100820000C942C040D3011F00C941904DC9A0C94E7
:100830002C040E3011F00C942004DD9A0C942C043E
:100840000F3011F00C942704DE9A0C942C04003124
:1008500011F00C942C04DF9A0091A100003111F0EA
:100860000C942103B3990C94690480E991E00E94EF
:10087000721FB3990C945404A9EAB0E08C9187FBE1
:1008800016F00C944A047091A9007F777093A90028
:100890000C944F047091A90070687093A900B39BE9
:1008A0000C944F040C9464040091A3000D3011F0DB
:1008B0000C945F0481E08093A3000C946404A3EA89
:1008C000B0E08C918F5F8C937091A90070647093ED
:1008D000A90083E083BF8F918FBFFF91EF91DF91DC
:1008E000CF91BF91AF919F918F917F916F915F91C8
:1008F0004F913F912F911F910F91BF90AF907F909B
:100900005F904F903F902F901F900F901895000090
:1009100000000000000000000000000000000000D7
:1009200000000000000100000000000000000001C5
:1009300000000000000100000000000000000001B5
:1009400000000000000100000000000000010001A4
:100950000000000000010000010000000001000193
:100960000000000000010000010000000101010181
:100970000000000000010000010000000101010171
:100980000000000000010000010001000101010160
:10099000000000010001000001000100010101014F
:1009A000000000010001000001000101010101013E
:1009B000000001010001000001000101010101012D
:1009C000000001010001000001010101010101011C
:1009D000010001010001000001010101010101010B
:1009E00001000101000101000101010101010101FA
:1009F00001000101000101010101010101010101E9
:100A000001010101000101010101010101010101D7
:100A100001010101010101010101010101010101C6
:100A200001010101010101010101010101010101B6
:100A300001010101010001010101010101010100A8
:100A40000101010101000101010101010101010098
:100A50000101010101000101010101010100010089
:100A6000010101010100010100010101010001007A
:100A7000010101010100010100010101000000006C
:100A8000010101010100010100010101000000005C
:100A9000010101010100010100010001000000004D
:100AA000010101000100010100010001000000003E
:100AB000010101000100010100010000000000002F
:100AC0000101000001000101000100000000000020
:100AD0000101000001000101000000000000000011
:100AE0000001000001000101000000000000000002
:100AF00000010000010000010000000000000000F3
:100B000000010000010000000000000000000000E3
:100B100000000000010000000000000000000000D4
:100B200000000000000000000000000000000000C5
:100B300000000000000000000000000000000100B4
:100B400000000000000000000000000000000101A3
:100B50000000000000000000000000000000010193
:100B60000100000000000000000000000000010182
:100B70000101000000000000000000000000010171
:100B80000101000000010000000000000000010160
:100B9000010100000101000000000000000001014F
:100BA000010100010101000000000000000001013E
:100BB000010101010101000000000000000001012D
:100BC000010101010101010000000000000001011C
:100BD000010101010101010100000000000001010B
:100BE00001010101010101010100000000000101FA
:100BF00001010101010101010101000000000101E9
:100C000001010101010101010101000000010101D7
:100C100001010101010101010101000001010101C6
:100C200001010101010101010101000101010101B5
:100C300001010101010101010101010101010101A4
:100C40000101010101010101010101010101010194
:100C50000101010101000101010101010101010086
:100C60000101010101000101010101010101010076
:100C70000101010101000101010101010100010067
:100C80000101010101000101000101010100010058
:100C9000010101010100010100010101000000004A
:100CA000010101010100010100010101000000003A
:100CB000010101010100010100010001000000002B
:100CC000010101000100010100010001000000001C
:100CD000010101000100010100010000000000000D
:100CE00001010000010001010001000000000000FE
:100CF00001010000010001010000000000000000EF
:100D000000010000010001010000000000000000DF
:100D100000010000010000010000000000000000D0
:100D200000010000010000000000000000000000C1
:100D300000000000010000000000000000000000B2
:100D400000000000000000000000000000000000A3
:100D50000000000000000000000000000000010191
:100D60000101010101010101010101010101010173
:100D70000101010101010101010101010101010163
:100D80000101010101010101010101010101010153
:100D90000101010101010101010101010101000045
:100DA0000000000000000000000000000000000043
:100DB0000000000000000000000000000000000033
:100DC0000000000000000000000000000000000023
:100DD0000000000000000000000000000000000013
:100DE0000000000000000000000000000000000003
:100DF00000000000000000000000000000000000F3
:100E000000000000000000000000000000000101E0
:100E100001010101010101010101010101010101C2
:100E200001010101010101010101010101010101B2
:100E300001010101010101010101010101010101A2
:100E40000101010101010101010101010101000094
:100E50000000000000000000000000000000010190
:100E6000010100000000000000000000000001017E
:100E7000010101010101000000000000000001016A
:100E80000101010101010101010100000000010156
:100E90000101010101010101010101010101000044
:100EA0000000010101010101010101010101000036
:100EB000000000000000010101010101010100002A
:100EC000000000000000000000000101010100001E
:100ED0000000000000000000000000000000000012
:100EE00000000000000000000000010101010000FE
:100EF00000000000000001010101010101010000EA
:100F000000000101010101010101010101010101D3
:100F100001010101010101010101010101010101C1
:100F200001010101010101010101000000000101B5
:100F300001010101010100000000000000000101A9
:100F4000010100000000000000000000000000009F
:100F50000000000000000000000000000000000190
:100F60000203010203040203040303040302010257
:100F70000304000102030304030402030201020349
:100F8000040301000102040302030102010003043F
:100F90000302020100010302010200010001040337
:100FA000020103020100020100010100010203022B
:100FB0000100040302010100010002010203020119
:100FC0000001030403020001020103020304010003
:100FD00001020203040301020302040304030100EB
:100FE00000000001000000000100000000010001FD
:100FF00000000001000000000100000001000000EE
:1010000001000000010000010000000100000000DC
:1010100000010000010000010000010000000000CC
:1010200000000000010101010000000000000000BC
:1010300000000101000000000101000000000100AB
:1010400000000000000000000000000000000000A0
:101050000000000000000000000000000000000090
:101060000000000000000000000000000000000080
:10107000000000000000000000000000010000006F
:10108000000000000000000000000001000000005F
:101090000000000000000000000000000000000050
:1010A0000000000000000000000000000000000040
:1010B000000000000000000000000E000000000022
:1010C0000000000000000000000000000000000020
:1010D0000000000000000000000000000000000010
:1010E00000000000000001000000000000000000FF
:1010F00000000100000000000000000000000000EF
:1011000000000000000000000000000000000000DF
:1011100000000000000000000000000000000000CF
:1011200000000000000000000000000000010000BE
:1011300000000000000000000000000000000000AF
:10114000000000000000000000000000000000019E
:10115000000000000000000000000000000000008F
:10116000010000000000000000000000000000007E
:10117000000000000000000000000000000000006F
:10118000000000000000000000000000000000005F
:10119000000E000000000000000000000000000041
:1011A000000000000000000000000000000000003F
:1011B000000000000000000000000000000000002F
:1011C000000000000001000000000000000000001E
:1011D000000000000000000000010000000000000E
:1011E00000000000000000000000000000000000FF
:1011F00000000000000000000000000000000101ED
:1012000001010101010101010101010101010000D0
:1012100000000000000000000000000000000000CE
:1012200000000000000000000000000000000000BE
:1012300000000000000000000000000000000000AE
:10124000000000000000000000000000000000009E
:10125000000000000000000000000000000001018C
:101260000101010101010101010101010101000070
:10127000000000000000000000000000000001016C
:10128000010100000000000000000000000000005C
:10129000000001010101000000000000000000004A
:1012A000000000000000010101010000000000003A
:1012B000000000000000000000000101010100002A
:1012C000000000000000010101010000000000001A
:1012D0000000010101010000000000000000010108
:1012E00001010000000000000000000000000000FC
:1012F00000000000000000000000000000000100ED
:1013000000000100000001000000010000000001D9
:1013100000000001000000010000000100000000CA
:1013200001000000010000000100000001000000B9
:1013300000010000000100000001000000010000A9
:101340000100000001000000010000000100000198
:101350000000000100000001000000010000010089
:10136000000001000000010000000100000000007A
:10137000000000000000000000000000000000006D
:1013800000000000000000000C0C00000C0C00002D
:10139000000000000000000000000000000000004D
:1013A000000000000000000000000000000000003D
:1013B000000000000000000000000000000000002D
:1013C000000000000000000000000000000000001D
:1013D000000000000000000000000000000000000D
:1013E0000C0C00000C0C0000000000000000000CC1
:1013F0000C00000C0C0000000000000000000C0CB1
:1014000000000C0C000000000000000000000000C4
:1014100000000000000000000000000000000000CC
:1014200000000000000000000000000000000000BC
:1014300000000000000000000000000000000000AC
:10144000000000000000000000000000000000009C
:10145000000000000000000000000000000000008C
:101460000000000000000C0C00000C0C000000004C
:10147000000000000000000C0C00000C0C0001003B
:101480000000000000010000010000010000000158
:101490000000010000000000000100000100000049
:1014A0000100000100000100000000000001000038
:1014B0000001000001000001000001000000000028
:1014C0000001000001000001000001000000000018
:1014D0000100000100000100000000000001000107
:1014E00000000100000000000001000001000100F8
:1014F00000000000000100000100000100000100E8
:1015000000000000000100000100000100000001D7
:1015100000000100000000000001000001000000C8
:1015200001000001000001000000000000010000B7
:1015300000010000010000010000010000000000A7
:10154000000000000000000000000000000000009B
:10155000000000000000000000000000000100008A
:101560000000000000000000010000000001000079
:101570000000000001000000010000000001000068
:101580000000000001000000010000010001000057
:101590000001000001000000010000010001000145
:1015A0000001000001000000010000010001000135
:1015B0000101000001000000010000010001010123
:1015C0000101000001000000010000010001010113
:1015D0000101000001000000010001010001010102
:1015E00001010000010000000100010101010101F1
:1015F00001010001010000000100010101010101E0
:1016000001010001010001000100010101010101CE
:1016100001010001010001000101010101010101BD
:1016200001010101010001000101010101010101AC
:10163000010101010101010001010101010101019B
:10164000010101010101010101010101010101018A
:10165000010101010101010101010101010101017A
:10166000010101010101010101010101010001016B
:10167000010101010101010100010101010001015C
:10168000010101010001010100010101010001014D
:10169000010101010001010100010100010001013E
:1016A0000100010100010101000101000100010030
:1016B0000100010100010101000101000100010020
:1016C0000000010100010101000101000100000012
:1016D0000000010100010101000101000100000002
:1016E00000000101000101010001000001000000F3
:1016F00000000101000101010001000000000000E4
:1017000000000100000101010001000000000000D4
:1017100000000100000100010001000000000000C5
:1017200000000100000100010000000000000000B6
:1017300000000000000100010000000000000000A7
:101740000000000000000001000000000000000098
:101750000000000000000000000000000000000089
:101760000000000000000000000000000000010078
:101770000000000000000000000000000000010068
:101780000000010000000000000000000000010057
:101790000000010000000100000000000000010046
:1017A0000000010000000100000001000000010035
:1017B0000000010000000100000001010000010024
:1017C0000000010000000101000001010000010013
:1017D0000000010100000101000001010000010101
:1017E00000000101000001010000010100000101F1
:1017F00001000101000001010000010100000101E0
:1018000001000101010001010000010100000101CE
:1018100001000101010001010100010100000101BD
:1018200001000101010001010100010101000101AC
:10183000010001010100010101000101010101019B
:10184000010001010100010101010101010101018A
:101850000100010101010101010101010101010179
:101860000101010101010101010101010101010168
:101870000101010101010101010101010101010158
:101880000101010101010101010101010100010149
:10189000010101010101010100010101010001013A
:1018A000010101010001010100010101010001012B
:1018B000010101010001010100010100010001011C
:1018C000010001010001010100010100010001000E
:1018D00001000101000101010001010001000100FE
:1018E00000000101000101010001010001000000F0
:1018F00000000101000101010001010001000000E0
:1019000000000101000101010001000001000000D0
:1019100000000101000101010001000000000000C1
:1019200000000100000101010001000000000000B2
:1019300000000100000100010001000000000000A3
:101940000000010000010001000000000000000094
:101950000000000000010001000000000000000085
:101960000000000000000001000000000000000076
:101970000000000000000000000000000000000067
:101980000000000000000000000000000000000057
:101990000000000000000000000000000000010145
:1019A0000101010101010101010101010101010127
:1019B0000101010101010101010101010101010117
:1019C0000101010101010101010101010101010107
:1019D00001010101010101010101010101010000F9
:1019E00000000000000000000000000000000000F7
:1019F00000000000000000000000000000000000E7
:101A000000000000000000000000000000000000D6
:101A100000000000000000000000000000000000C6
:101A200000000000000000000000000000000101B4
:101A30000101010101010101010101010101010196
:101A40000101010101010101010101010101010186
:101A50000101010101010101010101010101010176
:101A60000101010101010101010101010101000068
:101A70000000000000000000000000000000000066
:101A80000000000000000000000000000000010154
:101A90000101000000000000000000000000010142
:101AA000010101010101000000000000000001012E
:101AB000010101010101010101010000000001011A
:101AC0000101010101010101010101010101000008
:101AD00000000101010101010101010101010000FA
:101AE00000000000000001010101010101010000EE
:101AF00000000000000000000000010101010000E2
:101B000000000000000000000000000000000000D5
:101B100000000000000000000000010101010000C1
:101B200000000000000001010101010101010000AD
:101B30000000010101010101010101010101010197
:101B40000101010101010101010101010101010185
:101B50000101010101010101010100000000010179
:101B6000010101010101000000000000000001016D
:101B70000101000000000000000000000000000063
:101B80000000000000000000000000000000000055
:101B9000020300020304020304030304030200021D
:101BA000030400000203030403040203020002030F
:101BB0000403000000020403020300020000030407
:101BC0000302020000000302000200000000040300
:101BD00002000302000002000000000000020302F5
:101BE00000000403020000000000020002030200E3
:101BF00000000304030200000200030203040000CB
:101C000000020203040300020302040304030001B0
:101C100000000001000000000100000001000000C1
:101C200001000000010000010000000100000000B0
:101C300000010000010000010000010000000000A0
:101C40000000000001010101000000000000000090
:101C5000000001010000000001010000000001007F
:101C60000000000100000000010000000001000071
:101C70000000000000000000000000000000000064
:101C80000000020000000000000000000000000052
:101C90000000000000000000000000000002000042
:101CA0000000000000000000000000000000000034
:101CB0000000000000000000000000000000000024
:101CC00000000000000000000000200000000000F4
:101CD0000000000000000200000000000000000002
:101CE00000000000000000000000000000000000F4
:101CF00000000000000000000000000200000000E2
:101D000000000000000000000000200000000000B3
:101D100000000000000000000000000000000000C3
:101D200000000000000000000000000000000200B1
:101D300000000000000000000000000000000000A3
:101D40000000000000000000000000000200000091
:101D50000000000000000000000000000000000083
:101D6000000000000000000000020000000002006F
:101D70000000000000000000000000000000000063
:101D80000000000000000000000000000000000053
:101D90000000000000000000000000000000000043
:101DA0000020000000000000000000000000000013
:101DB0000000000000020000000000000000000021
:101DC0000000000000000000000000000000000013
:101DD0000200000000000000000000000000000001
:101DE00000200000000000000000000000000000D3
:101DF00000000000000000000000000000000000E3
:101E000000000000000000000000000000000000D2
:101E100000000000000000000000000000020002BE
:101E200000000000000000000000000000000000B2
:101E300000000000000000000000000000000101A0
:101E40000101010101010101010101010101000084
:101E50000000000000000000000000000000000082
:101E60000000000000000000000000000000000072
:101E70000000000000000000000000000000010160
:101E80000101010101010101010101010101000044
:101E90000000000000000000000000000000000042
:101EA0000000000000000000000000000000010130
:101EB0000101000000000000000000000000000020
:101EC000000001010101000000000000000000000E
:101ED00000000000000001010101000000000000FE
:101EE00000000000000000000000010101010000EE
:101EF00000000000000001010101000000000000DE
:101F000000000101010100000000000000000101CB
:101F100001010000000000000000000000000000BF
:101F200000000000000000000000000000000100B0
:101F3000000001000000010000000100000000019D
:101F4000000000010000000100000001000000008E
:101F5000010000000100000001000000010000007D
:101F6000000100000001000000010000000100006D
:101F7000010000000100000001000000010000015C
:101F8000000000010000000100000001000001004D
:101F9000000001000000010000000100000000003E
:101FA0000000000000000000000000000000000031
:101FB00000000000000000000C0C00000C0C0000F1
:101FC00000000017170000171700000000000000B5
:101FD0000000000000000000000000000000000001
:101FE00000000000000000000000000000000000F1
:101FF00000000000000000000000000000000000E1
:102000000000001717000017170000000000000074
:102010000C0C00000C0C0000000000000000000C84
:102020000C00000C0C0000000000000000000C0C74
:1020300000000C0C00000000000000000000000088
:102040000000001717000017170000000000000034
:102050000000000000000000000000000000000080
:102060000000000000000000000000000000000070
:102070000000000000000000000000000000000060
:1020800000000017170000171700000000000000F4
:102090000000000000000C0C00000C0C0000000010
:1020A000000000000000000C0C00000C0C000002FE
:1020B000000002000000000000020000020000001A
:1020C0000200000200000200000000000002000008
:1020D00000020000020000020000020000000200F6
:1020E00000000000000200000200000200000000EA
:1020F00002000002000002000000000000020002D6
:1021000000000200000000000002000002000200C7
:1021100000000000000200000200000200000000B9
:1021200000020000020000020000020000000002A5
:102130000000020000000000000200000200000099
:102140000200000200000200000000000002000087
:102150000002000002000002000002000000020075
:102160000000000000020000020000020000000069
:10217000000000000000000000000000000000005F
:10218000000000000000000000000100000000004E
:10219000000000000001000000000100000000003D
:1021A000000000000001000000000100000100002C
:1021B000000000010001000000000100000100001B
:1021C0000000000100010000000001000101000109
:1021D00000000001000100000000010001010001F9
:1021E00000010001000100000000010001010001E8
:1021F00000010001000100000000010101010001D7
:1022000000010001000101000000010101010101C4
:1022100000010001000101000000010101010101B4
:1022200000010101000101000000010101010101A3
:102230000001010100010100000101010101010192
:102240000001010101010100000101010101010181
:102250000001010101010100010101010101010170
:10226000010101010101010001010101010101015F
:10227000010101010101010101010101010101014E
:10228000010101010101010101010101010101013E
:10229000010101010101010101010001010101012F
:1022A0000101010101000101010100010101010120
:1022B0000101010101000101010100010100010111
:1022C0000101010001000101010100010100010102
:1022D00001010100010001010101000100000100F4
:1022E00001010100010001010101000100000100E4
:1022F00001000100010001010101000100000100D5
:1023000001000100010001010101000000000100C5
:1023100001000100010000010101000000000000B7
:1023200001000100010000010101000000000000A7
:102330000100000001000001010100000000000098
:102340000100000001000001010000000000000089
:10235000010000000000000101000000000000007A
:10236000010000000000000100000000000000006B
:10237000000000000000000100000000000000005C
:10238000000000000000000000000000000000004D
:10239000000000000000000000000000000000003D
:1023A000000000000000000000000000000100002C
:1023B000000000000000000000010000000100001B
:1023C000000000000001000000010000000100000A
:1023D00000010000000100000001000000010000F9
:1023E00001010000000100000001000000010000E8
:1023F00001010000010100000001000000010000D7
:1024000001010000010100000101000000010000C5
:1024100001010000010100000101000001010000B4
:1024200001010000010100000101000101010000A3
:102430000101000001010001010100010101000092
:102440000101000101010001010100010101000180
:10245000010100010101000101010001010101016F
:10246000010100010101000101010001010101015F
:10247000010101010101000101010001010101014E
:10248000010101010101010101010001010101013D
:10249000010101010101010101010101010101012C
:1024A000010101010101010101010101010101011C
:1024B000010101010101010101010001010101010D
:1024C00001010101010001010101000101010101FE
:1024D00001010101010001010101000101000101EF
:1024E00001010100010001010101000101000101E0
:1024F00001010100010001010101000100000100D2
:1025000001010100010001010101000100000100C1
:1025100001000100010001010101000100000100B2
:1025200001000100010001010101000000000100A3
:102530000100010001000001010100000000000095
:102540000100010001000001010100000000000085
:102550000100000001000001010100000000000076
:102560000100000001000001010000000000000067
:102570000100000000000001010000000000000058
:102580000100000000000001000000000000000049
:10259000000000000000000100000000000000003A
:1025A000000000000000000000000000000000002B
:1025B000000000000000000000000000000000001B
:1025C000000000000000000000000000000000000B
:1025D00000000000000000000000000000000101F9
:1025E00001010101010101010101010101010101DB
:1025F00001010101010101010101010101010101CB
:1026000001010101010101010101010101010101BA
:1026100001010101010101010101010101010000AC
:1026200000000000000000000000000000000000AA
:10263000000000000000000000000000000000009A
:102640000000000000000000000000000000010188
:10265000010101010101010101010101010101016A
:10266000010101010101010101010101010101015A
:10267000010101010101010101010101010101014A
:10268000010101010101010101010101010100003C
:10269000000000000000000000000000000000003A
:1026A000000000000000000000000000000000002A
:1026B0000000000000000000000000000000010118
:1026C0000101000000000000000000000000010106
:1026D00001010101010100000000000000000101F2
:1026E00001010101010101010101000000000101DE
:1026F00001010101010101010101010101010000CC
:1027000000000101010101010101010101010000BD
:1027100000000000000001010101010101010000B1
:1027200000000000000000000000010101010000A5
:102730000000000000000000000000000000000099
:102740000000000000000000000001010101000085
:102750000000000000000101010101010101000071
:10276000000001010101010101010101010101015B
:102770000101010101010101010101010101010149
:10278000010101010101010101010000000001013D
:102790000101010101010000000000000000010131
:1027A0000101000000000000000000000000000027
:1027B0000000000000000000000000000000000019
:1027C00000030000030400030403030403000000EB
:1027D00003040000000303040304000300000003DB
:1027E00004030000000004030003000000000304D1
:1027F00003000000000003000000000000000403CC
:1028000000000300000000000000000000000300C2
:1028100000000403000000000000000000030000AE
:102820000000030403000000000003000304000094
:10283000000000030403000003000403040300007D
:102840000100000001000001000000010000000084
:102850000001000001000001000001000000000074
:102860000000000001010101000000000000000064
:102870000000010100000000010100000000010053
:102880000000000100000000010000000001000144
:102890000000000100000000010000000100000035
:1028A0000000000000000000000000000000000028
:1028B0000000000000000000000000000300030012
:1028C0000000000000000000000000000000000008
:1028D00000000000000000000000000000000000F8
:1028E00000000000000000000000000000000000E8
:1028F00000000000000000000000200000000000B8
:1029000000000000000000000000000300000000C4
:1029100000000000000000000000000000000000B7
:1029200000000000000003000000000000000000A4
:102930000000000000000000000020000000000077
:102940000000000000000000000000000000000087
:102950000000000000000000000000000000000077
:102960000000000000000000000000000003000064
:102970000000030000000000000000000000000054
:102980000000000000000000000000000000000344
:102990000000000000000000000000000000000037
:1029A0000000000000000000000000000003000024
:1029B0000000000000000000000000000000000017
:1029C0000000000000000000000000000000000007
:1029D00000200000000000000000000000000000D7
:1029E00003000000000000000000000000000000E4
:1029F00000000000000000000000000000000000D7
:102A000000000000000300000000000000000000C3
:102A10000020000000000000000000000000000096
:102A200000000000000000000000000000000000A6
:102A30000000000000000000000000000000030093
:102A40000000000000000000000000000000000086
:102A50000000000000000000000300000000000073
:102A60000000000000000000000000000000000066
:102A70000000000000000000000000000000010154
:102A80000101010101010101010101010101000038
:102A90000000000000000000000000000000010134
:102AA0000101010101010101010101010101000018
:102AB0000000000000000000000000000000000016
:102AC0000000000000000000000000000000000006
:102AD00000000000000000000000000000000101F4
:102AE00001010000000000000000000000000000E4
:102AF00000000101010100000000000000000000D2
:102B000000000000000001010101000000000000C1
:102B100000000000000000000000010101010000B1
:102B200000000000000001010101000000000000A1
:102B3000000001010101000000000000000001018F
:102B40000101000000000000000000000000000083
:102B50000000000000000000000000000000010074
:102B60000000010000000100000001000000000161
:102B70000000000100000001000000010000000052
:102B80000100000001000000010000000100000041
:102B90000001000000010000000100000001000031
:102BA0000100000001000000010000000100000120
:102BB0000000000100000001000000010000010011
:102BC0000000010000000100000001000000000002
:102BD00000000000000000000000000000000000F5
:102BE00000000000000000000000000000000000E5
:102BF0000000001717000017170000000000222235
:102C00000000222200000000000000000000000080
:102C1000000022220000222200000000000000002C
:102C2000000000000000222200002222000000001C
:102C30000000001717000017170000000000000038
:102C40000000000000000000000000000000000084
:102C50000000000000000000000000000000000074
:102C60000000000000000000000000000000000064
:102C700000000017170000171700000000000000F8
:102C800000000000000000002222000022220000BC
:102C900000000000222200002222000000000000AC
:102CA000222200002222000000000000000000009C
:102CB00000000017170000171700000000000000B8
:102CC0000000000000000000000000000000000004
:102CD00000000000000000000000000000000000F4
:102CE00003000003000003000000000000030000D8
:102CF00000030000030000030000030000000300C5
:102D000000000000000300000300000300000003B7
:102D100000000300000000000003000003000003A7
:102D20000000030000000000000300000300030097
:102D3000000000000003000003000003000000008A
:102D40000003000003000003000003000000000077
:102D50000300000300000300000000000003000067
:102D60000300000300000300000000000003000057
:102D70000003000003000003000003000000030044
:102D80000000000000030000030000030000000337
:102D9000000003000000000000030000030000002A
:102DA0000000000000000000000000000000010022
:102DB0000000000000000000000000000000010012
:102DC0000000000000000000010000000000010001
:102DD00000000000000000000100000001000100F0
:102DE00000000001000000000100000001000100DF
:102DF00000000001000001000100000001000100CE
:102E000000000001010001000100000001000100BC
:102E100000000001010001000100010001000100AB
:102E20000000010101000100010001000100010199
:102E30000000010101000100010001000100010189
:102E40000000010101000101010001000100010178
:102E50000000010101000101010001000101010167
:102E60000001010101000101010001000101010156
:102E70000001010101010101010001000101010145
:102E80000001010101010101010001010101010134
:102E90000101010101010101010001010101010123
:102EA0000101010101010101010101010101010112
:102EB0000101010101010101010101010101000103
:102EC00001010101010101010101010101010001F3
:102ED00001010101010101010001010101010001E4
:102EE00001010101010101010001010100010001D5
:102EF00001010100010101010001010100010001C6
:102F000001010100010100010001010100010001B6
:102F100001010100000100010001010100010001A7
:102F20000101010000010001000100010001000198
:102F3000010100000001000100010001000100008A
:102F4000010100000001000100010001000100007A
:102F5000010100000001000000010001000100006B
:102F6000010100000001000000010001000000005C
:102F7000010000000001000000010001000000004D
:102F8000010000000000000000010001000000003E
:102F9000010000000000000000010000000000002F
:102FA0000000000000000000000100000000000020
:102FB0000000000000000000000000000000000011
:102FC0000000000000000000000000000000000001
:102FD00000000000000000000000000000010000F0
:102FE00000000000000000000000000001010000DF
:102FF00000000000000000000000000101010000CE
:1030000000000000000000000000010101010000BC
:1030100000000000000001000000010101010000AB
:10302000000000000000010100000101010100009A
:103030000000000000000101010001010101000089
:103040000000000000000101010101010101000078
:103050000000000000010101010101010101000067
:103060000000000001010101010101010101000056
:103070000000000101010101010101010101000045
:103080000000010101010101010101010101010033
:103090000000010101010101010101010101010122
:1030A0000000010101010101010101010101010112
:1030B0000100010101010101010101010101010101
:1030C00001010101010101010101010101010101F0
:1030D00001010101010101010101010101010001E1
:1030E00001010101010101010101010101010001D1
:1030F00001010101010101010001010101010001C2
:1031000001010101010101010001010100010001B2
:1031100001010100010101010001010100010001A3
:103120000101010001010001000101010001000194
:103130000101010000010001000101010001000185
:103140000101010000010001000100010001000176
:103150000101000000010001000100010001000068
:103160000101000000010001000100010001000058
:103170000101000000010000000100010001000049
:10318000010100000001000000010001000000003A
:10319000010000000001000000010001000000002B
:1031A000010000000000000000010001000000001C
:1031B000010000000000000000010000000000000D
:1031C00000000000000000000001000000000000FE
:1031D00000000000000000000000000000000000EF
:1031E00000000000000000000000000000000000DF
:1031F00000000000000000000000000000000000CF
:1032000000000000000000000000000000000000BE
:1032100000000000000000000000000000000101AC
:10322000010101010101010101010101010101018E
:10323000010101010101010101010101010101017E
:10324000010101010101010101010101010101016E
:103250000101010101010101010101010101000060
:10326000000000000000000000000000000001015C
:10327000010101010101010101010101010101013E
:10328000010101010101010101010101010101012E
:10329000010101010101010101010101010101011E
:1032A0000101010101010101010101010101000010
:1032B000000000000000000000000000000000000E
:1032C00000000000000000000000000000000000FE
:1032D00000000000000000000000000000000000EE
:1032E00000000000000000000000000000000101DC
:1032F00001010000000000000000000000000101CA
:1033000001010101010100000000000000000101B5
:1033100001010101010101010101000000000101A1
:10332000010101010101010101010101010100008F
:103330000000010101010101010101010101000081
:103340000000000000000101010101010101000075
:103350000000000000000000000001010101000069
:10336000000000000000000000000000000000005D
:103370000000000000000000000001010101000049
:103380000000000000000101010101010101000035
:10339000000001010101010101010101010101011F
:1033A000010101010101010101010101010101010D
:1033B0000101010101010101010100000000010101
:1033C00001010101010100000000000000000101F5
:1033D00001010000000000000000000000000000EB
:1033E00000000000000000000000000000000000DD
:1033F00000000000000400000400000400000000C1
:1034000000040000000000040004000000000000B0
:1034100004000000000004000000000000000004A0
:103420000000000000000000000000000000040098
:10343000000000000000000000000000000000008C
:103440000000040000000000000000000000000078
:103450000000000400000000000000000004000064
:103460000000000004000000000004000400000050
:103470000001000001000001000001000000000048
:103480000000000001010101000000000000000038
:103490000000010100000000010100000000010027
:1034A0000000000100000000010000000001000118
:1034B0000000000100000000010000000100000009
:1034C00001000000010000010000000100000000F8
:1034D00000000000000000000000000000040000E8
:1034E00000000000000000000000000000000000DC
:1034F00000000000000000000000000000000000CC
:1035000000000400000000000000000000000000B7
:1035100000000000000004000000000000000000A7
:10352000000000000000000000000000000000009B
:10353000000000000000000000000000000000008B
:10354000000000000000000000000E00000000006D
:103550000000000000000000000000020000000069
:10356000000000000000000000000000000000005B
:103570000000000000000000000000040000000047
:103580000000000000000000000000000400000037
:10359000000000000000000000000000000000002B
:1035A0000000000000000000000000000000040017
:1035B000000000000000000000000000000000000B
:1035C00000000000000000000000000000000000FB
:1035D00000000000000000000000000000000000EB
:1035E00000000000000000000004000000000000D7
:1035F00000000000000400000000000000000000C7
:1036000000000000000000000000000000000000BA
:1036100000000000000000000000000000000000AA
:10362000000E00000000000000000000000000008C
:10363000000000000000000000000000000000008A
:10364000000000000000000000000000000000007A
:103650000400000000000000000000000000000462
:10366000000000000000000000000000000000005A
:10367000000000000000000000000000000000004A
:10368000000000000000000000000000000000003A
:10369000000000000000000000000000000000002A
:1036A000000000000000000000000000000000001A
:1036B0000000000000000000000000000000010108
:1036C00001010101010101010101010101010000EC
:1036D00000000000000000000000000000000000EA
:1036E00000000000000000000000000000000000DA
:1036F00000000000000000000000000000000000CA
:1037000000000000000000000000000000000101B7
:1037100001010000000000000000000000000000A7
:103720000000010101010000000000000000000095
:103730000000000000000101010100000000000085
:103740000000000000000000000001010101000075
:103750000000000000000101010100000000000065
:103760000000010101010000000000000000010153
:103770000101000000000000000000000000000047
:103780000000000000000000000000000000010038
:103790000000010000000100000001000000000125
:1037A0000000000100000001000000010000000016
:1037B0000100000001000000010000000100000005
:1037C00000010000000100000001000000010000F5
:1037D00001000000010000000100000001000001E4
:1037E00000000001000000010000000100000100D5
:1037F00000000100000001000000010000000000C6
:1038000000000000000000000000000000000000B8
:1038100000000000000000000000000000000000A8
:103820000000000000000000000000000000222254
:103830000000222200000000000000000000000044
:1038400000002222000022220000000000000000F0
:1038500000000000000022220000222200000000E0
:103860000000000000000000000000000000000058
:103870000000000000000000000000000000000048
:103880000000000000000000000000000000000038
:103890000000000000000000000000000000000028
:1038A0000000000000000000000000000000000018
:1038B0000000000000000000222200002222000080
:1038C0000000000022220000222200000000000070
:1038D0002222000022220000000000000000000060
:1038E00000000000000000000000000000000000D8
:1038F00000000000000000000000000000000000C8
:1039000000000000000000000000000000000000B7
:103910000004000004000004000004000000040093
:103920000000000000040000040000040000000487
:10393000000004000000000000040000040000007B
:103940000400000400000400000000000004040063
:10395000000000000004000004000004000000005B
:103960000004000004000004000004000000000047
:103970000400000400000400000000000004000433
:10398000000004000000000000040000040000002B
:103990000004000004000004000004000000040013
:1039A0000000000000040000040000040000000407
:1039B00000000400000000000004000004000000FB
:1039C00004000004000004000000000000040100E6
:1039D00000000000000000000000000000000101E5
:1039E00000000000000000000000000000000101D5
:1039F00001000000000000000000000000000101C4
:103A000001010000000000000000000000000101B2
:103A100001010000000100000000000000000101A1
:103A20000101000000010000000100000000010190
:103A3000010100000001000000010000000101017F
:103A4000010100000001000000010000010101016E
:103A5000010100000001000000010001010101015D
:103A6000010100000001000000010101010101014C
:103A7000010100000001010000010101010101013B
:103A8000010101000001010000010101010101012A
:103A90000101010100010100000101010101010119
:103AA0000101010101010100000101010101010108
:103AB00001010101010101000101010101010101F7
:103AC00001010101010101010101010101010001E7
:103AD00001010101010101010101010101010000D8
:103AE00001010101010101010101010101010000C8
:103AF00000010101010101010101010101010000B9
:103B000000000101010101010101010101010000A9
:103B1000000001010100010101010101010100009A
:103B2000000001010100010101000101010100008B
:103B3000000001010100010101000101010000007C
:103B4000000001010100010101000101000000006D
:103B5000000001010100010101000100000000005E
:103B6000000001010100010101000000000000004F
:103B70000000010101000001010000000000000040
:103B80000000000101000001010000000000000031
:103B90000000000001000001010000000000000022
:103BA0000000000000000001010000000000000013
:103BB0000000000000000001000000000000000004
:103BC00000000000000000000000000000000100F4
:103BD00000000000000000000000000000000101E3
:103BE00000000000000000000000000000000101D3
:103BF00001000000000000000000000000000101C2
:103C000001010000000000000000000000000101B0
:103C1000010100000001000000000000000001019F
:103C2000010100000001000000010000000001018E
:103C3000010100000001000000010000000101017D
:103C4000010100000001000000010000010101016C
:103C5000010100000001000000010001010101015B
:103C6000010100000001000000010101010101014A
:103C70000101000000010100000101010101010139
:103C80000101010000010100000101010101010128
:103C90000101010100010100000101010101010117
:103CA0000101010101010100000101010101010106
:103CB00001010101010101000101010101010101F5
:103CC00001010101010101010101010101010101E4
:103CD00001010101010101000101010101010101D5
:103CE00001010101010101000001010101010101C6
:103CF00001010101000101000001010101010101B7
:103D000001010100000101000001010101010101A7
:103D10000101000000010100000101010101010198
:103D20000101000000010000000101010101010189
:103D3000010100000001000000010001010101017A
:103D4000010100000001000000010000010101016B
:103D5000010100000001000000010000000101015C
:103D6000010100000001000000010000000001014D
:103D7000010100000001000000000000000001013E
:103D8000010100000000000000000000000001012F
:103D90000100000000000000000000000000010120
:103DA0000000000000000000000000000000010012
:103DB0000000000000000000000000000000000003
:103DC00000000000000000000000000000000100F2
:103DD00000010000000000000000010000010101DE
:103DE00001010100000101000001010101010101C7
:103DF00001010101010101010101010101010001B4
:103E000001000101010101010101000101000000A7
:103E1000000000010100000101000000000000009E
:103E20000000000000000000000000000000000092
:103E3000000001010000000001010000000000007E
:103E4000000000000101010100000000000000006E
:103E5000000100000100000100000100000000005E
:103E6000010000000100000100000001000000014D
:103E7000000000010000000001000000010001003E
:103E8000000000010000000001000000000105D05A
:103E90000E94811F00FC0CD008950024E89457FF75
:103EA00002C009D0689400F80BD010F801240895DE
:103EB00002D009D00895509540954F5F5F4F089507
:103EC000E89417FF0895009510950F5F1F4F6894B1
:103ED00008953197F1F70895689462F80895E89489
:103EE00062F80895EF93FF93EE27E82BE92B31F06A
:103EF000E6EAFEE03197F1F70197D1F7FF91EF91F4
:103F000008950F92B801469F8001479F100D569F5C
:103F1000100D0F900895C89531960020089591E0F6
:103F200005C092E003C094E001C098E0F4DF0D9278
:0C3F30009A95E1F70895E80FF91FF1CF12
:00000001FF
